:03000000021204E5
:03000B000200C12F
:03002B000203EBE2
:03005B0002053D5E
:0300730002053350
:1000800002030406080C10182030406080020304AC
:1000900006080C101820304080FF0406080C1018C9
:1000A0002030406080A0C000000001010003020277
:1000B000010D0D040506020D0505050D06040502DA
:1000C00002C2AFC0D0C0E0205A0D302F02E473301E
:1000D000600280F90203D7306306C2B1C287C281D1
:1000E00085258AC25AE525F4700221CA056130606F
:1000F00013206A19758B00D0E0D0D0C2B1C287C27C
:1001000081D2AF32C2B1C287C2810201BAD26EC2FD
:100110006FE565601CC3E5611495654014C26ED23D
:100120006FC3E561956450030201BA756100020175
:10013000BA206C14C2B1C287C2817406D5E0FDD268
:1001400082D286D2800201BAD26FC2B1C287C28186
:10015000E53D20E23420E1127406D5E0FD20750271
:10016000D280307502D2820201BA20E0127406D524
:10017000E0FD207502D280307502D2820201BA748D
:1001800006D5E0FDD2860201BA20E11F20E00A7404
:1001900006D5E0FDD2860201BA7406D5E0FD2075D1
:1001A00002D282307502D2800201BA7406D5E0FD17
:1001B000207502D282307502D280758B00D0E0D0DB
:1001C000D0C2B1C287C281D2AF32D0E0D0D0D2AFDC
:1001D0003261D7E525600A207502D2B1307502D2AE
:1001E00081C28761D7E5256002D287207502C2816E
:1001F000307502C2B161D7E525600A207502D2814F
:10020000307502D2B1207502C2B1307502C281616F
:10021000D7207502C282307502C280E525600A20AF
:100220007502D2B1307502D281207502C28030755C
:1002300002C282C28761D7207502C282307502C2B3
:1002400080207502C280307502C2827406D5E0FD3E
:10025000E525600A207502D2B1307502D281C287CD
:1002600061D7207502C282307502C280E525600A1E
:10027000207502D2B1307502D281C286C28761D7A1
:10028000207502C282307502C280C2867406D5E033
:10029000FDE525600A207502D2B1307502D281C217
:1002A0008761D7C286E5256002D287207502C282A7
:1002B000307502C280207502C281307502C2B16100
:1002C000D7C286207502C282307502C2807406D5FC
:1002D000E0FDE5256002D287207502C281307502FB
:1002E000C2B161D7C286E5256002D287207502C2FD
:1002F00080307502C282207502C281307502C2B19F
:1003000061D7C286207502C280307502C28274062F
:10031000D5E0FDE5256002D287207502C2813075E7
:1003200002C2B161D7207502C280307502C282E577
:1003300025600A207502D281307502D2B1C28620B2
:100340007502C2B1307502C28161D7207502C280C8
:10035000307502C282C2867406D5E0FDE525600ACA
:10036000207502D281307502D2B1207502C2B1303F
:100370007502C28161D7207502C280307502C282C7
:10038000E525600A207502D281307502D2B1207550
:1003900002C282307502C280207502C2B13075027D
:1003A000C28161D7207502C280307502C282207579
:1003B00002C282307502C2807406D5E0FDE5256078
:1003C0000A207502D281307502D2B1207502C2B105
:1003D000307502C28161D7E525F4F58A758B007509
:1003E0006000D25AD0E0D0D0D2AF32C2AFC0D0C0BD
:1003F000E0D2D3C2CEE528600A741F552E6049159D
:1004000028814878007900E580307601F430E502F3
:1004100078FF53DACF20760343DA2030760343DACD
:1004200010C2D8C269E580307601F430E50279FF68
:10043000C3E89970CE305903752818741F552E6083
:10044000037528188858D268E52960041529815B4E
:10045000741F552E600543DA01C2D820680281ED71
:10046000E558F8C268741F552E60367982B704319A
:0F047000C3E894F0400374F0F8E8C4540F28F880
:10047F007984B7030281A1C313C313872120080214
:10048F00C313200A06C3C898F881A128F850037433
:10049F00FFF8C3E8955F5003E55FF8E52C5406704D
:1004AF003D882230630AC3E522955C4003855C22B8
:1004BF007882B60429C3E5229524401278A096408D
:1004CF000DE52426F52450097524FF0204E085224A
:1004DF0024852425C3E524955C4003855C2520CF26
:1004EF0009D0E0D0D0C2D3D2AF32C2CF7801E52845
:1004FF006008741F552E70021528C3E558940140EB
:10050F0005755B00A11CE55B046002055BE55DC33F
:10051F00240A5005755DFFA12AF55DD0E0D0D0C249
:10052F00D3D2AF32C2AF53917FC258D2AF32C2AF24
:10053F00C0D0C0E0C0F0D2D3A8FBA9FCC2D83069AC
:10054F0002A1A053DACF20760343DA1030760343AB
:10055F00DA20D269E580307601F420E502A17488B3
:10056F00268927E14053DACF20760343DA2030760D
:10057F000343DA10C2D8C269741F552E7002E126E8
:10058F007800E580307601F430E502E1268858E105
:10059F002653DACF20760343DA2030760343DA107E
:1005AF00C269205902C15A53DACF20760343DA10B9
:1005BF0030760343DA20C2D8D26988538954C3E80E
:1005CF009551F8E99552F9E4FB7AFAC3E894C8E932
:1005DF0094005008E4D2E4FB7A0AC12DC3E8946872
:1005EF00E994015008E4D2E3FB7A0FC12DC3E894DC
:1005FF00D0E994025008E4D2E2FB7A1EC12DC3E881
:10060F0094A0E994055008E4D2E1FB7A3CC12DC3D4
:10061F00E89498E994085006E4D2E0FB7A78C3E8AE
:10062F009555FCE99556FD30E708ECF42401FCEDF7
:10063F00F4FD7557007008C3EC9A50037557018885
:10064F00558956A853A95488518952C3E89526F85D
:10065F00E99527F9307402C1F9307302C1F930728C
:10066F0002C1F2E9C313F9E813F8307102C1F2E9DC
:10067F00C313F9E813F8307002C1F2E9C313FDE8B0
:10068F0013FC205918C3EC941CED9402400302078D
:10069F0026ED7009C3EC94C8500302074074002084
:1006AF0077037896E624FAFEE43400FFC3EC9EFC51
:1006BF00ED9FFD500678007900C1F9C3EC94FFED72
:1006CF009400400678FF7900C1F9EC856CF0A4C561
:1006DF00F0A2F733F87900400302071578FF79008D
:1006EF00020715E9C313F9E813F830740EE9600235
:1006FF0078FFC3E81338F8E43400F9C3E894FFE94E
:10070F009400400278FF8858D268205902E126747D
:10071F001FF4552E4BF52E752818741F552E700388
:10072F0075280A305902E140741F552E600353DAC1
:10073F00FE752906741F552E700375290AD0F0D047
:10074F00E0D0D0C2D3D2AF327901E16F7903E16F3C
:10075F00790AE16F791EE16F7964E16F79C8E16F12
:10076F007817E4D5E0FDD8FAD9F6227A147B78020F
:10077F0007967A107B8C0207967A0D7BB402079648
:10078F007A0B7BC8020796AC257525017902B275E5
:10079F00E4C286D5E0FDE5256002D287D5E0FDC233
:1007AF0087D5E0FDD286D5E0FDE525600A207502EC
:1007BF00D2B1307502D281E56DD5E0FD207502C250
:1007CF00B1307502C2817496D5E0FDD9C1EAF8D572
:1007DF00E0FDD8FBDBB1C2868C2522C37C007D00F7
:1007EF0075F00005F0EA33FAEB33FB50F6EB13FB31
:1007FF00EA13FAC3E9FFE8FEE89AF8E99BF9500417
:10080F00EFF9EEF8B3EC33FCED33FDD5F0DFEDF996
:10081F00ECF822E889F08A20D2D4F8A9F07B0030D6
:10082F00F70B7BFFF42401F8E9F43400F9E8852095
:10083F00F0A4ADF0F8E98520F0A4AFF0FEED2EF9AD
:10084F0074003FFA7C04C3EA13FAE913F9E813F8CA
:10085F00DCF48BF030F70AE8F42401F8E9F4340003
:0F086F00F9E889F0C2D4F8A9F0227882B6040320
:10087E000208D6C3E5589401400302089E8522243F
:10088E00E4F53FF540F541F542F543F5480208D64B
:10089E007882E6FC754801E522F523783879C7AAF7
:1008AE003BAB3CC3EB13FBEA13FAEC146013C3EB44
:1008BE0013FBEA13FAEC14146007C3EB13FBEA13F1
:1008CE00FA1207EA883F894022E5486034C3E53FC3
:1008DE009523F8E5409400F9500CC3E89480E99410
:1008EE00FF401602090BC3E8947FE99400500302FF
:1008FE00090B787F790002090B788079FF8844898B
:10090E004522E5486058E5442541F8E5453542F96C
:10091E00854520E4300701F43543FA30E709C3EA90
:10092E0094F0401502094DC3EA940F500302094D8D
:10093E0078FF79FF7A0F02094D780079007AF0C3BB
:10094E00E524955C5006E52460092166E54520E71F
:10095E000D2166E54530E706884189428A4322E546
:10096E004870030209D0789EE6FAC3E54433F8E5F1
:10097E004533F91122E930E70BC3E89480E994FF7F
:10098E00401321A7C3E8947FE99400500221A77871
:10099E007F790021A7788079FFE820E715C3E5234A
:1009AE0098F84009C3E8940140030209CE78010289
:1009BE0009CEE8F424012523F840030209CE78FF7E
:1009CE00884622E5487003020A32789FE6FAA8426A
:1009DE00A9431122E930E70CC3E89401E994FF40E2
:1009EE0016020A09C3E894FFE994005003020A09AB
:1009FE0078FF7900020A09780179FFE920E715C32B
:100A0E00E54698F84009C3E894014003020A30789D
:100A1E0000020A30E8F424012546F84003020A30A9
:100A2E0078FF8824227883E6F520120F6F75E89000
:100A3E00E5E820ECF0A8BDA9BE1210047568557546
:100A4E006900C3740013FD745513FC74552CFC74AB
:100A5E00003DFDECFAEDFBC3E89AE99B4014E56816
:100A6E002455F568E5693400F569EA2CFAEB3DFB8F
:100A7E0080E5AE68AF69C3E56913F9E56813F8C39D
:100A8E00E913F9E813F8E56828F566E56939F567BD
:100A9E007A03C3E913F9E813F8DAF7AA201A7009F2
:100AAE00756800756900020AC71AEA6008EE28FE2A
:100ABE00EF39FFDAF88E688F692275E89022788315
:100ACE00E6FFE5E820ECF7A8BDA9BE056AC3E56A16
:100ADE0094084052756A00E97007E56B601B020AC4
:100AEE00FBC3E8956B6010E56B5006600C14020BAF
:100AFE00070460F9020B07E56BF56BC394A8F84089
:100B0E0021755CC0C3E89405F84017755C80C3E896
:100B1E009405F8400D755C40C3E89405F8400375E4
:100B2E005C0075BB0622EFC39401601BC3E894FF03
:100B3E00E994035012C3E89568E995695009E55C9C
:100B4E00600C155C020B5CE55CF46002055CA85C55
:100B5E00C3E524985002A8248825C3E525955D4059
:100B6E000B855D25E55DF46003855D5CC3E56AB4C8
:100B7E00070375BB1E22306102783230620278782C
:100B8E00E52C5406601FE879A187F0A4C5F0A2F702
:100B9E0033F8C3E8955C4002A85C88228824882537
:100BAE00306102885E22788FE6FFC3EF94055018FD
:100BBE00C3EF94045020C3EF94035028C3EF940264
:100BCE005030C3EF940150387533A075340F75351E
:100BDE003C753605811C7533C075341275354075FC
:100BEE003606811C7533707534177535D07536071A
:100BFE00811C75334C75341D7535C4753609811CD1
:100C0E007533287534237535B875360B811C8533CD
:100C1E004F853450753B00753C0822A84FA95002F1
:100C2E000C34A849A94A759100C3E498F594E49947
:100C3E00F595759104D25875C820A8CCA9CD75C864
:100C4E0024AA39AB3A8839893AC3E89AF8E99BF96C
:100C5E00AA3BAB3CC3EB13FDEA13FCC3ED13FDEC57
:0F0C6E0013FCC3EA9CFAEB9DFBEA28FAEB39FB77
:100C7D008A3B8B3C400122753BFF753CFF2230586F
:100C8D0002818B759100C3E4954BF594E4954CF579
:100C9D0095759104D258227892E6FF7E10305B0252
:100CAD007F053063047F037E00A93CA83B7A04C313
:100CBD00E913F9E813F8DAF7C3E89EF8E99400F9B7
:100CCD004009C3E89402E9940050047802E4F9E97C
:100CDD00FBE8FAC3E913FDE813FCC3EF9403602EA0
:100CED00EF20E00DE82CF8E93DF9ECFAEDFB020DF3
:100CFD0008E828F8E939F97A02E4FBC3EF940340D8
:100D0D000D8A4D8B4E8849894A8C4B8D4C22884DCE
:100D1D00894E8A498B4A8C4B8D4C22305802A12822
:100D2D00759100C3E4953BF594E4953CF59575916B
:100D3D0004D25822753E00752000020D50753E00FC
:100D4D00752040D2AF053E20580122759D00E53C2F
:100D5D00C313C313F8086030306A06C313C313F806
:100D6D0008C3E8940A4002780A306D08C3E8940479
:100D7D0040027804C3E53C9408400D759D02C3E51F
:100D8D003C94104003759D03205803D2AF22791E69
:100D9D00206D02790AD2AF0000C2AF205A0A793C09
:100DAD00206D027914306FE03063027978C3E58BE2
:100DBD009920630240F740D0E59BF45440B52002E2
:100DCD00A150D8C4D2AF22C25B789CE6146007E56F
:100DDD003E147002D25B30630B0538205810753805
:100DED0000020DFB2058071581158102175F227532
:100DFD009100C3E4954DF594E4954EF595759104E8
:100E0D00D25822AE25305B4F78A3E6FFBF010BD23F
:100E1D005C752500C2B1C287C2819190305C0375AB
:100E2D002500305802C129BF020BD25C752500C2C6
:100E3D00B1C287C28178A2B6010D9190305C037565
:100E4D002500305802C149BF030BD25C752500C285
:100E5D00B1C287C281B1FC305C03752500305802E8
:100E6D00C164305B04C25C8E2522C2AFC286206A8B
:100E7D0003020E9690034B306E0F207502C2803028
:100E8D007502C2827406D5E0FD207502D2823075DE
:100E9D0002D280759F02753D02D2AF22C2AF206A89
:100EAD0003020ECB900302306E17C286207502C26C
:100EBD0080307502C2827406D5E0FD020ECE90011F
:100ECD00E5207502C281307502C2B1305A06E525A2
:100EDD006002D287207503759F03307503759F01DE
:100EED00753D03D2AF22C2AF207502C282307502AA
:100EFD00C280206A03020F129002C1306E07C286B3
:100F0D007406D5E0FD207502D280307502D28220A4
:100F1D007503759F01307503759F03753D04D2AF41
:100F2D0022C2AF206A03020F50900280306E17204C
:100F3D007502C282307502C280C2867406D5E0FD8C
:100F4D00020F539001D3C287305A0EE525600A2057
:100F5D007502D2B1307502D281759F02753D05D2F1
:100F6D00AF22C2AF207502C280307502C282206AE4
:100F7D0003020F96900237306E0F207502C2823039
:100F8D007502C2807406D5E0FDD286207503759F6B
:100F9D0003307503759F01753D06D2AF22C2AF2098
:100FAD006A03020FD49003A4306E1F207502C28213
:100FBD00307502C280207502C280307502C2827403
:100FCD0006D5E0FD020FD79001F7207502C2B130B2
:100FDD007502C281305A0EE525600A207502D28154
:100FED00307502D2B1207503759F01307503759F61
:100FFD0003753D01D2AF229001D1C2B1C287C2812A
:10100D00C282C286C28022C3E54F9535E550953622
:10101D005001227890E6FFC3EF94055018C3EF946A
:10102D0004501BC3EF9403501EC3EF94025021C311
:10103D00EF94015024C3E54F943CF802106FC3E5C3
:10104D004F9428F802106FC3E54F941AF802106FF1
:10105D00C3E54F9412F802106FC3E54F940AF802DE
:0F106D00106FE5509400F9884F895022305803D6
:10107C00021079227880760778817607788276015B
:10108C00788476037883760178867609788F760172
:10109C00789076057895760278927603789B760D23
:1010AC007893760678877601789C76027888760134
:1010BC007889760178857600788C7601788D760043
:1010CC00788E76B478967625789776D078987678E8
:1010DC00789976C8789A7604789D7600227893E68B
:1010EC00FF756409756501C3BF02097564057565F3
:1010FC000102112EC3BF0309756405756502021147
:10110C002EC3BF040975640575650302112EC3BF98
:10111C000506756409756507C3BF06067564007519
:10112C0065007887E6FFC26CC3BF0302D26CC26B4A
:10113C00C3BF0402D26BC26A7418552D6002D26A06
:10114C00C26E6002D26ED26F6002C26FC2757888B6
:10115C00E630E102D275C2767889E630E102D276C9
:10116C00C3EF94026008758E01D26D02117F758EEB
:10117C0000C26D227880E61490008093789EF678F9
:10118C0081E61490008093789FF6110422789BE6F8
:10119C001490008D9378A0F61104227886E61490B2
:1011AC00009A9378A1F6110422789CE6149000A77B
:1011BC009378A2F6789CE6149000AC9378A3F61181
:1011CC000422C2B3789DE66002D2B3227896E6FA86
:1011DC007897E6FB3077047A007BFFC3EB9AFCC36D
:1011EC00948250027C82756C00056CEC856CF0A4CA
:1011FC00C3E5F0948040F222C2D353D9BF7581C0AD
:10120C0043FF8012075775EF0243B203E5B3240482
:10121C004002F5B375803875A4C775F1FF75D4DF3E
:10122C007590FF75A50075F20075D50075A0FF755A
:10123C00A60075F30075D60075B0E475A71B75F4A0
:10124C00FF75E2411104E4F8F6D8FD118012178DF8
:10125C0011E93180319931A731B531CE31D8789837
:10126C00866D110475885075890275C824759104B2
:10127C0075D84012076B12077A1207631207811296
:10128C000763120788120763121CE512076B12071B
:10129C006B12076775A82275B80275E69075F61083
:1012AC00759B80759D0375D10E75BC5875BB067505
:1012BC00BA1F75E880120757D2AF120A3343DA010E
:1012CC00C2D8C26912076B753001D2597A05E5573D
:1012DC0070027A0512075BE558C3940240EEE52EC6
:1012EC00541F855A59F55AB559E2DAE2C25953DA04
:1012FC00CF20760343DA2030760343DA10C2D8C20B
:10130C006912076712075B7802741F552E700278FA
:10131C0000C3E5589840EDC2AF12077A12077A1253
:10132C00077AD2AF12076B75470012075B788CE611
:10133C00C3940150030213FFE530C3940150030220
:10134C0013FF741F552E6035C3E55894FF500302EC
:10135C0013FFC2AF12078FD2AF120767C3E55894C1
:10136C000150EFC2AF12077A12075F12077AD2AFA1
:10137C00120767C3E55894FF40E9021D6A7F05D246
:10138C007731D8120767C2AFC27731D8C3E558940A
:10139C007FD2AF4068C2AF12078FD2AFDFE1C3E597
:1013AC005894057897F612076B12183C121CED7FB7
:1013BC000AD27731D8120767C2AFC27731D8C3E5EA
:1013CC0058947FD2AF50E8C2AF12077A12075F125F
:1013DC00077AD2AFDFDBE55824057896F612076B57
:1013EC0012183C121D1C120767C3E55894FF40F6F7
:1013FC00021D6AC3E5589547400385584712076795
:10140C00C3E558940140026136C2AF12078F120730
:10141C008F12078FD2AF12076B753000E4F531F5E0
:10142C00320531E531F470360532789AE6782814B5
:10143C006012785014600D78A014600878F0146075
:10144C0003753200C3E53298401415327899866DD5
:10145C00C2AF12078FD2AF7898866D12076712074A
:0E146C005BE5287008741F552E700241D6C330
:10147A00E558940640AD120767E52870030212D6B4
:10148A001104E4F522F523F524F525755CFF78852A
:10149A00865FF53FF540F541F542F543F56AF548B3
:1014AA00F52BF52CF55B120BB4756A0875BB1E1289
:1014BA000757120AC8E5E820ECFBA8BDA9BEE970E7
:1014CA0001F8886B120ACC756A0875BB1E7895E616
:1014DA0030E00302151C7887E6FE760211E9788768
:1014EA00EEF6D261C2AF120B8485225C85225DD2F0
:1014FA00AFC261752500756200756301D260D2635F
:10150A00753800120F6F120FAA120C30120BB402A8
:10151A0016457887E6FE76037893E6FD760511E9A7
:10152A007887EEF67893EDF6D260D261D26E120F1A
:10153A006F120FAA120B84120757120E771207574F
:10154A00120757120EA912075B120EF312075B124B
:10155A00075B120F2E12075F120F6F12075B12073B
:10156A0057C261D262120AC8120ACC120B84756A77
:10157A000875BB1E120FAA120C29120CA411141101
:10158A0079120E77120C29120CA411141179120E69
:10159A00A9120C29120CA411141179120EF3120CAF
:1015AA0029120CA411141179120F2E120C29120CE3
:1015BA00A411141179120F6F120C29120CA4111410
:1015CA00C3E54F9535E5509536400C1179C3E5587A
:1015DA009401509102175F1179C2627887E6FE760C
:1015EA000211E97887EEF685225C855E5D855E25C7
:1015FA00756200756301D263753800C2AF20750247
:10160A00C282307502C280207502C280307502C261
:10161A0082742DD5E0FDD2AF120FAA120C30120C33
:10162A008B120CA4120D28756A0075BB06021645AA
:10163A0011E9120FAA756A0075BB06120D4A120D3E
:10164A00D4120DFC120879120E10120E77120C30F9
:10165A00120C8B120CA4120D28120D41120DD41269
:10166A000DFC1208D7120E10120EA9120C30120C11
:10167A008B120CA4120D28120D4A120DD4120DFC55
:10168A00120910120E10120EF3120C30120C8B12D9
:10169A000CA4120D28120D41120DD4120DFC1209C0
:1016AA006D120E10120F2E120C30120C8B120CA48B
:1016BA00120D28120D4A120DD4120DFC1209D11264
:1016CA000E10120F6F120C30120C8B120CA4120D8A
:1016DA0028120D41120AC8120DD4120DFC120ACC9E
:1016EA00120E10120FAA120C30120C8B120CA4122A
:1016FA000D2830632A855E5C855E5D7562007563C0
:10170A0001C3E5389464400AC263D264753714028F
:10171A001729C3E5589401400302164502175F30A2
:10172A006419E537147005C26402163AF537C3E541
:10173A00589401400302164502175FC3E55B94FA09
:10174A005013741F552E7004E5286009C3E53C94B4
:10175A00F05002C14511047887E6FE760211E97855
:10176A0087EEF6E4F522F523F524F525F55FC26048
:10177A001207571104741F552E7006E5287002418E
:10178A00D68128901A0D7820121C00E520B4550C39
:10179A00A3121C00E520B4AA030217AE1180121886
:1017AA003C02183B901A037880121C00A308121CF2
:1017BA0000A308121C00901A067883121C00A308C2
:1017CA00121C00A308A308121C00A308121C00A3E1
:1017DA0008121C00A308121C00A308A308A30812DD
:1017EA001C00A308A308121C00A308121C00A308CB
:1017FA00121C00A308A308121C00A308121C00A3B1
:10180A0008A308121C00A308121C00A308121C003B
:10181A00A308121C00A308121C00A308121C00A390
:10182A0008121C00A308121C00A308121C00901A1C
:10183A002122C2AF121C3F121C19901A00740A12FC
:10184A001C05A37404121C05A37410121C05901A1B
:10185A00037880121C04A308121C04A308121C0497
:0F186A00901A067883121C04A308121C04A3080A
:10187900A308121C04A308121C04A308121C04A325
:1018890008121C04A308A308A308121C04A308A394
:1018990008121C04A308121C04A308121C04A308A0
:1018A900A308121C04A308121C04A308A308121CF1
:1018B90004A308121C04A308121C04A308121C0484
:1018C900A308121C04A308121C04A308121C04A3D5
:1018D90008121C04A308121C04121C52121C30907A
:0318E9001A21229F
:101A00000A04100909040103FF0901010155AA0193
:101A1000FFFF0105FF0306FF0225D02850040D0239
:021A200000FFC5
:101A4000235475726E6967794145343541232020EE
:101A500023424C48454C4923463331302320202033
:101A60002020202020202020202020202020202076
:101C0000E493F622E6438F01538FFD75EF0275B71B
:101C1000A575B7F1F0538FFE22438F02438F0175F4
:101C2000EF0275B7A575B7F1901A0DF0538FFC222E
:101C3000901A0D74559105901A0E74AA9105227A86
:101C40003079D07820901A409100E520F709A3DA86
:101C5000F7227A3079D0901A40E7910509A3DAF992
:101C600022AB6EA86FBB01057980021CE2BB0205A6
:101C70007981021CE2BB03057982021CE2BB0405E8
:101C80007984021CE2BB05057983021CE2BB0605D0
:101C90007995021CE2BB07057986021CE2BB0805A8
:101CA000798F021CE2BB09057990021CE2BB0A0590
:101CB0007992021CE2BB0B05799B021CE2BB0C056E
:101CC0007993021CE2BB0D057987021CE2BB0E056D
:101CD000799C021CE2BB0F057988021CE27989021B
:101CE0001CE2E8F7227C0512076BDCFB22C2AF1274
:101CF000077A12078112078812078F12075F1207EF
:101D00007A12078112078812078F12075F12077A6B
:101D100012078112078812078FD2AF22C2AF1207B3
:101D20008F12078812078112077A12075F12078F36
:101D300012078812078112077A12075F12078F12A3
:101D4000078812078112077AD2AF22AE6EAF6FC238
:101D5000AF12077A12077A12077A12075FDEF212C1
:101D6000078F12075FDFF8D2AF2291ED91E591E581
:101D7000756E01756F01757000B14B7C05AD581221
:101D8000076BC3ED955870F5C3E55894014009C33E
:101D9000E55894FF4032A1A6916112183C91EDC222
:101DA000AF75EF1291E5DCD50570C3E57094035073
:101DB0000280C691E5056FE56E149000B193F808B6
:101DC000C3E56F98500280AE91E591E5056EC3E5DD
:101DD0006E94115002809C12108012183CC2AF7594
:041DE000EF1291E588
:00000001FF
